:100000000C9464040C948C040C948C040C948C0458
:100010000C948C040C948C040C948C040C94661E2C
:100020000C948C040C948C040C948C040C948C0410
:100030000C948C040C945B0E0C948C040C948C0427
:100040000C94551A0C948C040C948C040C948C0411
:100050000C948C040C948C040C948C040C948C04E0
:100060000C948C040C948C04C70BCD0BD80BDE0BBA
:10007000EC0BFC0B130CEA0CED0CF00CF30CF60C77
:10008000F90CFC0C110D1F0D280D360D440D500DF3
:10009000680D07634236B79BD8A71A39685618AE61
:1000A000BAAB558C1D3CB7CC5763BD6DEDFD753EAD
:1000B000F6177231BF000000803F00000000003ED4
:1000C0005B4F5B3E3E6B4F6B3E1C3E7C3E1C183CC8
:1000D0007E3C181C577D571C1C5E7F5E1C00183C24
:1000E0001800FFE7C3E7FF0018241800FFE7DBE76D
:1000F000FF30483A060E2629792926407F05050754
:10010000407F05253F5A3CE73C5A7F3E1C1C0808AF
:100110001C1C3E7F14227F22145F5F005F5F060974
:100120007F017F006689956A606060606094A2FFCD
:10013000A29408047E040810207E201008082A1CBF
:1001400008081C2A08081E101010100C1E0C1E0C8B
:1001500030383E3830060E3E0E060000000000002B
:10016000005F00000007000700147F147F14242A9A
:100170007F2A12231308646236495620500008076C
:100180000300001C2241000041221C002A1C7F1C8D
:100190002A08083E0808008070300008080808088F
:1001A000000060600020100804023E5149453E00F6
:1001B000427F400072494949462141494D33181454
:1001C000127F1027454545393C4A494931412111A3
:1001D00009073649494936464949291E0000140095
:1001E00000004034000000081422411414141414B8
:1001F000004122140802015909063E415D594E7C16
:100200001211127C7F494949363E414141227F41CA
:1002100041413E7F494949417F090909013E414128
:1002200051737F0808087F00417F41002040413F13
:10023000017F081422417F404040407F021C027F22
:100240007F0408107F3E4141413E7F090909063E77
:100250004151215E7F091929462649494932030146
:100260007F01033F4040403F1F2040201F3F403858
:10027000403F631408146303047804036159494D33
:1002800043007F4141410204081020004141417F69
:1002900004020102044040404040000307080020DF
:1002A000545478407F2844443838444444283844DF
:1002B00044287F385454541800087E090218A4A416
:1002C0009C787F0804047800447D40002040403D35
:1002D000007F1028440000417F40007C04780478AF
:1002E0007C080404783844444438FC182424181842
:1002F000242418FC7C08040408485454542404049E
:100300003F44243C4040207C1C2040201C3C40308A
:10031000403C44281028444C9090907C4464544CB9
:100320004400083641000000770000004136080014
:1003300002010204023C2623263C1EA1A161123ABE
:100340004040207A3854545559215555794121540B
:10035000547841215554784020545579400C1E5210
:1003600072123955555559395454545939555454B4
:10037000580000457C410002457D420001457C401B
:10038000F0292429F0F0282528F07C545545002038
:1003900054547C547C0A097F4932494949323248D5
:1003A000484832324A4848303A4141217A3A42403C
:1003B0002078009DA0A07D39444444393D40404010
:1003C0003D3C24FF2424487E4943662B2FFC2F2BE1
:1003D000FF0929F620C0887E090320545479410082
:1003E00000447D413048484A32384040227A007A01
:1003F0000A0A727D0D19317D2629292F28262929DF
:10040000292630484D402038080808080808080800
:10041000382F10C8ACBA2F102834FA00007B000027
:1004200008142A142222142A1408AA005500AAAA81
:1004300055AA55AA000000FF00101010FF00141468
:1004400014FF001010FF00FF1010F010F01414142F
:10045000FC001414F700FF0000FF00FF1414F40464
:10046000FC141417101F10101F101F1414141F0059
:10047000101010F0000000001F101010101F1010BE
:100480001010F010000000FF1010101010101010CD
:1004900010FF10000000FF140000FF00FF00001F0D
:1004A00010170000FC04F414141710171414F404AB
:1004B000F40000FF00F714141414141414F700F7D8
:1004C000141414171410101F101F141414F4141003
:1004D00010F010F000001F101F0000001F1400009B
:1004E00000FC140000F010F01010FF10FF141414A2
:1004F000FF141010101F00000000F010FFFFFFFF9E
:10050000FFF0F0F0F0F0FFFFFF0000000000FFFF41
:100510000F0F0F0F0F38444438447C2A2A3E147EB4
:1005200002020606027E027E026355494163384498
:10053000443C04407E201E2006027E020299A5E76C
:10054000A5991C2A492A1C4C7201724C304A4D4D07
:10055000303048784830BC625A463D3E49494900EF
:100560007E0101017E2A2A2A2A2A44445F4444400B
:10057000514A444040444A51400000FF0103E0809A
:10058000FF000008086B6B083612362436060F0988
:100590000F06000018180000001010003040FF0186
:1005A00001001F01011E00191D1712003C3C3C3CBC
:1005B000000000000000007A430000FA4300803B86
:1005C0004400007A4400409C440080BB4400C0DAF0
:1005D000440000FA4423282D32373C410A0014001D
:1005E0001E00280032003C00460050005A00640003
:1005F0006E00780082008C009600A000AA00B40073
:10060000BE00C80005000A0014001E0028003200C9
:10061000589E2CCF72DF96E778ECB9EF0DF2CBF352
:1006200026F53CF61FF7DDF77DF806F97DF9E6F9CA
:1006300041FA93FADCFA1EFB0A141E28323C46509B
:100640005A646E78828C96A0AAB4BEC864009600E4
:10065000C800FA002C015E019001000000000000BB
:10066000000000000000000000000000000000008A
:10067000000000000000000000000000000000007A
:10068000000000000000000000000000000000006A
:10069000000000000000000000000000000000005A
:1006A000000000000000000000000000000000004A
:1006B00000000000000003800400000000000000B3
:1006C0000003F01C000000000000000003FFFFE03A
:1006D0000000000000000003FFFE0000000000001A
:1006E000000003FFFF000000000000000003FFFE09
:1006F000C00000000000000001FFFF20000000001B
:1007000000000001FFFE800000000000000001FF6B
:10071000FE000000000000000001FFFE00000000DD
:100720000000000001FFFC000000000000000000CD
:10073000FFFC000000000000000000FFFF80000040
:100740000000000000007FFF00000000000000002B
:10075000007FFE00000000000000003EFFF80000E7
:10076000000000000000FF8FE0000000000000001B
:1007700000FF9FF00000000000000001FFFFF800F4
:1007800000000000000003FFFFF800000000000070
:100790000003FFFFF80000000000000007FFFFFC5F
:1007A0000000000000000007FFFFFE000000000046
:1007B000000007FFFFFE000000000000000FFFFF29
:1007C000FC000000000000000FF9EFE00000000056
:1007D0000000005FE01FF8000000000000007FE064
:1007E0003FFE000000000000007FC07FFF8000008F
:1007F000000000003F807FFFE00000000000001FBD
:10080000007FFFE00000000000000000000000008A
:1008100000000000000000000000000000000000D8
:1008200000000000000000000000000000000000C8
:1008300000000000000000000000000000000000B8
:1008400000000000000000000000000000000000A8
:100850000000000000000000000000000000000098
:10086000000000000000000000000000000800027E
:100870000100000304070000000000000000010266
:10088000040810204080010204081020010204081E
:1008900010200404040404040404020202020202FC
:1008A00003030303030300000000230026002900C4
:1008B00000000000250028002B000000000024009C
:1008C00027002A000200461A11241FBECFEFD8E0ED
:1008D000DEBFCDBF14E0A0E0B1E0ECEAF4E402C07A
:1008E00005900D92A834B107D9F725E0A8E4B4E04B
:1008F00001C01D92AE36B207E1F718E0C8ECD8E0AF
:1009000004C02297FE010E940022C63CD107C9F70D
:100910000E94C51E0C9454220C9400002F923F920A
:100920004F925F926F927F928F929F92AF92BF92FF
:10093000CF92DF92EF92FF920F931F93CF93DF93AB
:1009400000D000D0CDB7DEB74C017C836B836A0149
:100950005901C8018701AC014C195D0957FF03C05B
:1009600051954195510995016B817C81261B370B6F
:1009700037FF03C031952195310922242394312C6E
:100980002417350714F0212C312C2114310459F08F
:100990003A2D2B2D5C01832F922F3B812C81DC8201
:1009A000CB82C32ED22EAB81BC81AA16BB065CF4CF
:1009B0003C2D2D2D6C01832F922F3B812C81BC82ED
:1009C000AB82A32EB22E2501EB81FC814E1A5F0A69
:1009D0003C016C187D0877FE03C071946194710826
:1009E000720157FE03C0FFEFEF1AFF0AF594E79478
:1009F000C816D9062CF421E030E03A83298324C0BC
:100A00006FEF7FEF7A8369831FC0D401ED91FC9172
:100A10000480F581E02D980121143104D9F04B8137
:100A20005C81B601C4010995E618F708F7FE06C017
:100A3000E981FA81CE0EDF1EE40CF51C2B813C818E
:100A40002F5F3F4F3C832B836B817C81A616B706BB
:100A5000E4F604C0A6016B817C81E4CF0F900F9077
:100A60000F900F90DF91CF911F910F91FF90EF901A
:100A7000DF90CF90BF90AF909F908F907F906F90BE
:100A80005F904F903F902F9008956F927F928F923A
:100A90009F92AF92BF92CF92DF92EF92FF920F930D
:100AA0001F93CF93DF93EC015B016A013901480189
:100AB000E881F9810284F385E02D87010995E881B9
:100AC000F981A601480D591D415051090284F38551
:100AD000E02D9301B501CE010995E881F9810084EB
:100AE000F185E02D9401A601B501CE010995E881BB
:100AF000F981B501660D771D615071090084F1859A
:100B0000E02D9401A601CE010995DF91CF911F91AF
:100B10000F91FF90EF90DF90CF90BF90AF909F909C
:100B20008F907F906F900895EF92FF920F931F9395
:100B3000DC01ED91FC91240F351F21503109068015
:100B4000F781E02D780189019B0109951F910F9193
:100B5000FF90EF900895EF92FF920F931F93DC01A7
:100B6000ED91FC91260F371F215031090680F78146
:100B7000E02D78018A0109951F910F91FF90EF9068
:100B800008956F927F928F929F92AF92BF92CF9271
:100B9000DF92EF92FF920F931F93CF93DF935C014D
:100BA0004A0169013801EB01C60ED71ECC15DD05DF
:100BB00074F4D501ED91FC910084F185E02D87015D
:100BC0009301A401BE01C50109952196EFCFDF91E4
:100BD000CF911F910F91FF90EF90DF90CF90BF903A
:100BE000AF909F908F907F906F900895EF92FF92BB
:100BF0000F931F93DC01ED91FC9111971A960D91C3
:100C00001C911B9718962D913C9119970684F78596
:100C1000E02D7B0140E050E060E070E009951F911D
:100C20000F91FF90EF9008950895FC0113821282B6
:100C300086E393E09183808375836483578346833F
:100C40007187608753874287158A158614861786B1
:100C5000168621E0248B8FEF9FEF938B828B918BF5
:100C6000808B268B08952F923F924F925F926F92C6
:100C70007F928F929F92AF92BF92CF92DF92EF922C
:100C8000FF920F931F93CF93DF93CDB7DEB72897D3
:100C90000FB6F894DEBF0FBECDBF5C011B015C83B5
:100CA0004B8329013701C801079697FD07969C01E0
:100CB000B3E035952795BA95E1F73A832983812CDE
:100CC000912CE12CF12CE614F7040CF048C01886A6
:100CD0001F82AB81BC81AE0DBF1DBE83AD832F8152
:100CE0003885201731079CF5EF81F885F7FD379699
:100CF000A3E0F595E795AA95E1F7E80DF91DE40D58
:100D0000F51DE491F0E08F81988587709927A0E820
:100D1000B0E002C0B595A7958A95E2F7EA23FB23D8
:100D2000EF2B79F0D501ED91FC910480F581E02D58
:100D300096014D815E816F817885620D731DC501BD
:100D40000995EF81F8853196F887EF83C8CF3FEF9B
:100D5000E31AF30A89819A81880E991EB4CF2896E6
:100D60000FB6F894DEBF0FBECDBFDF91CF911F91BC
:100D70000F91FF90EF90DF90CF90BF90AF909F903A
:100D80008F907F906F905F904F903F902F9008953D
:100D90002F923F924F925F926F927F928F929F928B
:100DA000AF92BF92CF92DF92EF92FF920F931F9379
:100DB000CF93DF93CDB7DEB72C970FB6F894DEBF95
:100DC0000FBECDBF9C878B873A0118870F83FA86A9
:100DD000E986CD82DC0118968D919C911997681750
:100DE00079070CF094C01A968D919C911B97481727
:100DF00059070CF08CC08C2C912CCB01B6E0CB9E0B
:100E0000800D911D1124181619060CF080C0C40124
:100E100013E0880F991F1A95E1F7840F951F181694
:100E200019060CF074C0F5E02F9F200111245B011E
:100E30006B011C82920126543F4F2901461A570A22
:100E40003C81353031F0F201EA0DFB1D44914B83BA
:100E500001C01B827A82698213011E828B8180FF0E
:100E600013C0AB85BC85ED91FC91BD81B13031F4EF
:100E70000480F581E02D2F81388519C00684F7851F
:100E8000E02DEF80F8841EC0E985FA852F81388532
:100E9000E217F307F9F0AB85BC85ED91FC91BD81BC
:100EA000B13059F40480F581E02D29853A85A101FE
:100EB000B5018B859C8509950DC00684F785E02DCD
:100EC000E984FA848401940149815A81B6018B85B1
:100ED0009C850995EB81E695EB83FE81FF5FFE83A0
:100EE00029813A81280D391D3A8329833FEF231A3E
:100EF000330AF83009F0B2CF4C814F5F4C83C80CF5
:100F0000D91C8FEFA81AB80A463009F099CF2C9651
:100F10000FB6F894DEBF0FBECDBFDF91CF911F910A
:100F20000F91FF90EF90DF90CF90BF90AF909F9088
:100F30008F907F906F905F904F903F902F9008958B
:100F4000CF92EF92FF920F931F93CF93DF93EC0119
:100F5000262F6A3049F42C898E859F8538E0239F9F
:100F6000800D911D112432C06D30A1F1EA88FB88FB
:100F7000088919894E855F856C857D85CC880E949E
:100F8000C8062C89422F50E08C859D8536E0239F32
:100F9000800D911D11249D878C872E892223D1F0ED
:100FA0006AEF64039001659F300D1124688579858F
:100FB000260F371F281739076CF403E0440F551F1D
:100FC0000A95E1F78E859F85840F951F9F878E87F1
:100FD0001D861C8681E090E0DF91CF911F910F91DB
:100FE000FF90EF90CF900895FC0175876487578735
:100FF00046870895611101C061E0FC01648B08958A
:10100000FC01738B628B718B608B08956435710565
:10101000B0F54033510598F5CA01E3E09595879501
:10102000EA95E1F747705527232BA1F024E5289F87
:10103000F001299FF00D1124E60FF71FE050FF4F3C
:1010400081E090E0042E01C0880F0A94EAF79081B5
:10105000982B14C024E5289FF001299FF00D11243E
:10106000E60FF71FE050FF4F81E090E0042E01C033
:10107000880F0A94EAF780959081982390830895C9
:10108000CF92DF92EF92FF920F931F93CF93DF9354
:101090001F92CDB7DEB76C01162FF42E40E350E05F
:1010A00064E570E029830E9415068EE493E0F60162
:1010B00091838083F78A108F2981218FE28E038F9D
:1010C0000F90DF91CF911F910F91FF90EF90DF90E4
:1010D000CF900895FC0188E090E030E8A68DB78DB0
:1010E0004C9125A1209524232C93A48DB58D24A16A
:1010F000432F462321F04C91422B4C9304C04C913A
:10110000209524232C93A68DB78D2C9145A1242BBB
:101110002C933695019711F708951F93CF93DF9382
:10112000EC01162F60E0898D0E949E1B8B8D181696
:101130001CF460E00E949E1B612FCE010E946A0891
:101140008B8D181634F461E0DF91CF911F910C94D0
:101150009E1BDF91CF911F9108951F93CF93DF9333
:10116000EC01162F67FD1FE761E2CE010E948D089A
:10117000612F6068CE010E948D0860E2CE01DF9190
:10118000CF911F910C948D08DF92EF92FF920F93F5
:101190001F93CF93DF93EC01F0E0EF2EF1E0FF2EF1
:1011A000D12C6D2D6064CE010E948D0860E8CE01C7
:1011B0000E948D0861E0898D0E949E1B8B8D181600
:1011C0001CF460E00E949E1B00E010E0F701E00FBD
:1011D000F11F6081CE010E946A080F5F1F4F043526
:1011E0001105A1F78B8D18161CF461E00E949E1B5F
:1011F000D39484E5E80EF11C86E0D812D2CF60E4E7
:10120000CE01DF91CF911F910F91FF90EF90DF9072
:101210000C948D081F93CF93DF93EC01162F61E0A0
:101220008F890E94651B61E0888D0E94651B61E0CB
:10123000898D0E94651B8A8D18161CF461E00E943E
:10124000651B8B8D18161CF461E00E94651B8A8D4E
:10125000181684F460E00E949E1B2FEF89E698E147
:10126000215080409040E1F700C0000061E08A8D8D
:101270000E949E1B888D992787FD9095FC01EE5654
:10128000F74FE491F0E0EE0FFF1FE055F74F259187
:1012900034913F8F2E8FFC01E258F74F84918DA33C
:1012A0008F89992787FD9095FC01EE56F74FE491C1
:1012B000F0E0EE0FFF1FE055F74F259134913D8F81
:1012C0002C8FFC01E258F74F84918CA38B8D9927CA
:1012D00087FD9095FC01EE56F74FE491F0E0EE0F9C
:1012E000FF1FE055F74F2591349139A328A3FC0146
:1012F000E258F74F84918EA3898D992787FD9095A9
:10130000FC01EE56F74FE491F0E0EE0FFF1FE055C1
:10131000F74F259134913BA32AA3FC01E258F74FE4
:1013200084918FA361E2CE010E948D0864E1CE0119
:101330000E948D0817FD1FE7612F6068CE010E9493
:101340008D0860E2CE010E948D086CE0CE010E9403
:101350008D08CE01DF91CF911F910C94C40828EF26
:1013600031E0E0E0F1E0DF01A9011D924150504081
:10137000E1F7DC011D961C921E921C971F961C9291
:101380001E921E9708950C942E220C94362283E010
:101390008093B0008CE08093B1001092B300089568
:1013A0002F923F924F925F926F927F928F929F9275
:1013B000AF92BF92CF92DF92EF92FF920F931F9363
:1013C000CF93DF93CDB7DEB72E970FB6F894DEBF7D
:1013D0000FBECDBF3C014A015B0139872887180148
:1013E000EA8620E030E0A901C501B4010E943A1F5D
:1013F00087FD05C060E070E080E09FE304C060E02E
:1014000070E080E09FEB00E010E02885398502174E
:1014100013074CF420E030E040E251E40E943E1F0C
:101420000F5F1F4FF2CF9B01AC01C501B4010E94B9
:10143000D61E6B017C0120E030E0A901C501B4019A
:101440000E943A1F87FF04C0F7FAF094F7F8F0946F
:10145000412C512C3DEC39838CEC8D839CEC9E838C
:10146000EDE3EF8320E030E040E251E469817D81EB
:101470008E819F810E9453218B018D879B87A701BD
:1014800096010E943A1F181654F0FFEF4F1A5F0A98
:1014900009831D832D852E833B853F83E3CF411434
:1014A000510421F082010F5F1F4F02C002E010E0E3
:1014B00020E030E0A901C501B4010E943A1F87FF76
:1014C00002C00F5F1F4F888599850196800F911F7D
:1014D000EFEF2E1A3E0A8215930594F4281A390A62
:1014E000121413047CF4FA85FF2361F0F301C101A7
:1014F000860D971D20E22193E817F907E1F705C053
:10150000212C312C00E010E001C0810120E030E00E
:10151000A901C501B4010E943A1F87FF07C0F3016A
:10152000E00FF11F8DE280830F5F1F4F41145104C4
:1015300039F4F301E00FF11F80E380830F5F1F4F49
:101540001E861D869301200F311F3C872B872D851A
:101550003E85241535050CF03FC029813D814E8123
:101560005F81C701B6010E943E1F0E94D71F4B0139
:101570005C016B857C858D859E85680F791F4AE0AF
:10158000C4010E940922B401882777FD8095982F15
:101590000E940A2029813D814E815F810E94532152
:1015A0009B01AC01C701B6010E94D51E6B017C01F5
:1015B00020E030E040E251E469817D818E819F81AD
:1015C0000E943E1F69837D838E839F83ED85FE8508
:1015D0003196FE87ED87BBCF57FE02C0412C512CC0
:1015E000040D151D88859985181619063CF4F3011C
:1015F000E00FF11F8EE280830F5F1F4FA12CB12CF3
:101600004301800E911E28853985A216B3066CF51C
:1016100020E030E040E251E4C701B6010E945321CE
:101620006B017C010E94D71F69837A838B839C8323
:10163000B4016A0D7B1D4AE089819A810E940922CA
:10164000E981FA81BF01882777FD8095982F0E9454
:101650000A209B01AC01C701B6010E94D51E6B0197
:101660007C01FFEFAF1ABF0ACECFC90137FF02C01E
:1016700080E090E0B801680F791F121413048CF415
:101680003A8531110EC0F301E60FF71F9F0140E2CA
:101690004193CF01821B930B82159305CCF3620D0E
:1016A000731D660D771DFB011082C3012E960FB6C8
:1016B000F894DEBF0FBECDBFDF91CF911F910F9188
:1016C000FF90EF90DF90CF90BF90AF909F908F9062
:1016D0007F906F905F904F903F902F90089583E59B
:1016E00094E00E94AF0983E594E00C94C408882339
:1016F00049F093E49093B0009CE09093B100809304
:10170000B30008950C94C7094F925F926F927F9235
:101710008F929F92AF92BF92CF92DF92EF92FF9201
:101720000F931F93CF93DF931F92CDB7DEB782E065
:101730000E94D41B6C0121E0812C912C00E010E070
:10174000E12CF12C222309F487C00E946F0B40E0AA
:1017500050E060E070E083E594E00E94F407E1145B
:10176000F10461F4F801EE0FFF1FE250FD4F6081BC
:10177000718183E594E00E94481C6AC0073011051E
:1017800008F066C0F801EC5CFF4F0C94FE21F401F8
:10179000EE0FFF1FE45BF94F16C0F401E85CF94F50
:1017A00064914AE050E083E594E00E940A1D50C035
:1017B000F401EE0FFF1FEC5FF94F05C0F401EE0FCF
:1017C000FF1FE452FA4F659174914AE050E083E5BF
:1017D00094E00E94281D3CC0F401E25FFC4F808130
:1017E000882319F062E673E002C065E673E083E5E2
:1017F00094E00E943B1C2CC094012B523A4F59019B
:10180000F90164914AE050E083E594E00E940A1DEA
:1018100083E594E00E94C408F501649183E594E0B7
:101820000E94AD0811C0F401EE0FFF1FEE0FFF1F65
:10183000EB54FA4F459155916591749122E030E057
:1018400083E594E00E942F1E83E594E00E94C40883
:1018500083E594E00E94C40882E00E94D41B5C01EE
:101860008C159D05E9F4CD2809F0C7C10E949F1A87
:101870006419750986099709603D774081059105CE
:1018800030F461E08FE00E949E1B60E005C060E0E4
:101890008FE00E949E1B61E080E10E949E1BADC113
:1018A0000E949F1ACD2801F59B01AC01241935092E
:1018B0004609570929013A0135E6431651046104E6
:1018C000710490F060E08FE00E949E1B60E080E178
:1018D0000E949E1B40ED441647E0540661047104CB
:1018E00030F0DD24D39401C0D12CC12C03C0D12C05
:1018F000CC24C3940E949F1A2B013C01C11003C049
:10190000D11058C07AC151E0E516F10449F00F5FDB
:101910001F4F0830110509F04AC000E010E047C031
:101920008FEF881A980A0115110529F497E0891696
:10193000910429F522C00130110529F4E4E18E1645
:101940009104E9F41AC00230110529F4F6E08F166B
:10195000910411F51FC00330110531F424E1821602
:10196000910409F04FC04CC00430110541F432E03D
:101970008316910409F046C043C0812C912C053098
:10198000110551F447E08416910409F086C0812CBA
:10199000912C83C0812C912C0630110599F558E0CB
:1019A0008516910409F091C0812C912C8EC0DD2008
:1019B00009F4A8C0E114F10441F50730110509F458
:1019C000A3C00730110508F0A3C0F801E55CFF4F84
:1019D0000C94FE218090FD0211C08090FC020EC08C
:1019E0008090FB020BC08090FA0208C080904904EE
:1019F00005C08090F90202C08090F802912C88C046
:101A0000812C912CDD2009F4FBC00730110508F072
:101A100085C0C8018E5B9F4F94013327FC010C9455
:101A2000FE218092FD02F901EE0FFF1FE45BF94FEA
:101A30008591949190935204809351046FC0809249
:101A4000FC02F901E85CF94FE491E0934E0466C0B2
:101A50008092FB02F901EE0FFF1FEC5FF94F8591B9
:101A6000949190934D0480934C0458C08092FA0254
:101A7000F901EE0FFF1FE452FA4F85919491909374
:101A80004B0480934A044AC080924904F901E25F02
:101A9000FC4F80818093100341C0DD2009F4B0C069
:101AA0008092F902F401FF27EB52FA4F64916093A0
:101AB000110383E594E00E94AD0883E594E00E9461
:101AC000C40821E005E010E02AC0DD2009F498C038
:101AD0008092F802F401FF27EE0FFF1FEE0FFF1FA9
:101AE000EB54FA4F85919591A591B491809313038E
:101AF00090931403A0931503B093160321E006E01E
:101B000010E00DC021E07AC021E0DD24D3940AC0AA
:101B100021E0D12CEE24E394F12C04C021E0D12C5F
:101B2000E12CF12C64E170E080E090E029830E94D8
:101B3000CE1A2981D11002C0650104CE0E946F0B1C
:101B400040E050E060E070E083E594E00E94F4073C
:101B500069E673E083E594E00E94481C83E594E025
:101B60000E94C4086091FD0282E090E00E94C509D5
:101B70006091FC0283E090E00E94C5096091FB0245
:101B800084E090E00E94C5096091FA0285E090E04F
:101B90000E94C5096091490486E090E00E94C50951
:101BA0006091F90287E090E00E94C5096091F80217
:101BB00088E090E00E94C50963E080E090E00E9428
:101BC000C50966E081E090E00E94C50968EC70E01C
:101BD00080E090E00F90DF91CF911F910F91FF90E7
:101BE000EF90DF90CF90BF90AF909F908F907F90BD
:101BF0006F905F904F900C94CE1A20E0D12C92CF32
:101C000021E090CFF89410928000E1E8F0E010829B
:101C100080914F04909150049093850080938400AC
:101C2000808182608083808181608083EFE6F0E044
:101C300080818160808378940895F894EFE6F0E0E5
:101C400080818160808378940895F894EFE6F0E0D5
:101C500080818E7F808378940895F894289A80916B
:101C60005104909152040E94F61A289880E090E066
:101C700020917A00206420937A0020917A0026FD3A
:101C8000FCCF209178004091790030E0342BFC01AA
:101C9000EE0FFF1FEC56FB4F31832083019620E0AF
:101CA00030912C03231710F42F5FFACF843691055F
:101CB000F9F6789408951F920F920FB60F9211249F
:101CC0002F923F924F925F926F927F928F929F924C
:101CD000AF92BF92CF92DF92EF92FF920F931F933A
:101CE0002F933F934F935F936F937F938F939F9324
:101CF000AF93BF93EF93FF93CF93DF93CDB7DEB74F
:101D00006C97DEBFCDBF80914F04909150049093AB
:101D100085008093840082E00E94D41B90935D052F
:101D200080935C0580915C0590915D05892B09F09D
:101D30002DC20E94250E0E949F1A6B017C0161E05A
:101D40008FE00E949E1B60E080E10E949E1B8091BC
:101D5000100381110E94C70964E670E080E090E002
:101D60000E94CE1A82E00E94D41B90935D0580935E
:101D70005C0580915C0590915D05892B09F56AE011
:101D800070E080E090E00E94CE1A82E00E94D41BB6
:101D900090935D0580935C050E949F1A6C197D09E4
:101DA0008E099F09613D77408105910510F360E040
:101DB0008FE00E949E1B61E080E10E949E1BD9CFB4
:101DC00064E670E080E090E00E94CE1A80915C05AD
:101DD00090915D05892B41F482E00E94D41B909381
:101DE0005D0580935C05F2CF60E08FE00E949E1B52
:101DF00060E080E10E949E1B0E949F1A6C197D0981
:101E00008E099F09603D77408105910558F08091CA
:101E10001203813021F0823029F481E001C082E098
:101E20008093120380911F0391E0892780931F0301
:101E300080911F03882309F45BC0109288041092DC
:101E4000890410928A0410928B04809112038130CD
:101E500081F41092800410928104109282041092F6
:101E600083041092900410929104109292041092A4
:101E7000930480911203823041F410928C041092EA
:101E80008D0410928E0410928F0410927F04109291
:101E90007E0488EC90E090937D0480937C0481E044
:101EA00080932C030E946F0B80911203813031F4D8
:101EB00066E773E083E594E00E943B1C8091120387
:101EC000823031F46BE773E083E594E00E943B1CC1
:101ED00060E873E083E594E00E943B1C83E594E0B6
:101EE0000E94C40860E08FE00E949E1B61E0EBC28C
:101EF0000E946F0B80911203813031F468E873E027
:101F000083E594E00E943B1C80911203823031F4FF
:101F10006BE873E083E594E00E943B1C6EE873E09D
:101F200083E594E00E943B1C809112038130B1F460
:101F300040919004509191046091920470919304A7
:101F4000E12C00E010E020E030E0CE0101960E949C
:101F5000D009BC0183E594E00E94481C80911203E3
:101F60008230B1F440918C0450918D0460918E04C4
:101F700070918F04E12C00E010E020E030E0CE0111
:101F800001960E94D009BC0183E594E00E94481CA0
:101F900061E973E083E594E00E943B1C60912803B3
:101FA000709129034AE050E083E594E00E94281DE7
:101FB00060EB73E083E594E00E943B1C60912A0390
:101FC00070912B034AE050E083E594E00E94281DC5
:101FD00065E973E083E594E00E943B1C60912C036B
:101FE0004AE050E083E594E00E94111D80911203C5
:101FF0008230A9F569E973E083E594E00E943B1C17
:1020000040911B0350911C0360911D0370911E03AE
:10201000E12C00E010E020E030E0CE0101960E94CB
:10202000D009BC0183E594E00E943B1C6EE773E09D
:1020300083E594E00E943B1C4091170350911803E4
:102040006091190370911A0320E030E0CE010196EF
:102050000E94D009BC0183E594E00E94481CE091F5
:102060002803F0912903AA24AA9423E0B22E3BE28C
:10207000232E312C80912A0390912B030197E8178E
:10208000F90708F017C23F012FEF621A720AD30155
:10209000AA0FBB1FAC56BB4F4D915C91809028039B
:1020A0009090290320912A0330912B03C09028039C
:1020B000D0902903DF01AA0FBB1FAC56BB4F4D9038
:1020C0005C90E0902803F0902903FE8AED8AE0906E
:1020D0002A03F0902B0300912803109129031A8FF3
:1020E000098F00915304109154041C8F0B8F1FE033
:1020F000149FC001159F900D1124B5010E94C821A5
:102100008101061B170B41E050E0481959094E0F99
:102110005F1F62E5649FC001659F900D11242F5FD2
:102120003F4F2C193D09B9010E94C8219B01AFE026
:10213000A49DC001A59D900D1124B5010E94C82148
:102140006101C61AD70A4D895E89E41BF50B52E579
:102150005E9FC0015F9F900D11246FEFE61AF60A93
:10216000498D5A8DE41AF50AB7010E94C821AB8D3A
:10217000BC8D1696ED91FC911797EE24E394F12C0B
:10218000A60183E594E00995F30174CF0E942D0E1A
:1021900080911F03882309F49DC080917C04909155
:1021A0007D04883C910509F095C080E090E0FC0139
:1021B000EE0FFF1FEC56FB4F208131812F3F334044
:1021C000F1F001968436910591F70E94250E0E9448
:1021D0006F0B6CE973E083E594E00E943B1C83E5A0
:1021E00094E00E94C4088AE80E94770B68EE73E0CE
:1021F00080E090E00E94CE1A0E94C709FFCFFC0148
:10220000EE0FFF1FEC56FB4F208131812F3F3340F3
:1022100079F501968436910591F70E94250E0E946A
:102220006F0B63EA73E083E594E00E943B1C83E557
:1022300094E00E94C4088AE80E94770B68EE73E07D
:1022400080E090E00E94CE1A0E94C70964EF71E01E
:1022500080E090E00E94CE1A8AE80E94770B68EE38
:1022600073E080E090E00E94CE1A0E94C709FFCF81
:102270008230910540F09C012250310930932903AE
:102280002093280309C0109229031092280304C048
:1022900001968436910551F0FC01EE0FFF1FEC56BC
:1022A000FB4F208131812333310590F79C01215070
:1022B000310930932B0320932A0320912C03283CCF
:1022C00048F48B35910530F080912C038F5F80931B
:1022D0002C03E3C22091280330912903A1E060E0A0
:1022E00070E0CB0140912A0350912B03241735074E
:1022F00000F5A901440F551FFA01EC56FB4F019060
:10230000F081E02DEF3FF34039F0AA2329F061502E
:102310007C4F8F4F9F4F0AC0FA01EC56FB4F408114
:102320005181640F751F811D911DA0E02F5F3F4FEC
:10233000D9CF0E9408206B017C018091120381306B
:1023400081F48091880490918904A0918A04B091CD
:102350008B048093840490938504A0938604B093A7
:102360008704609188047091890480918A04909117
:102370008B04209124033091250340912603509132
:1023800027030E945321A70196010E94D61E609345
:1023900088047093890480938A0490938B048091BD
:1023A0001203813009F04CC0609120037091210329
:1023B0008091220390912303209180043091810425
:1023C0004091820450918304E0902003F090210317
:1023D0000091220310912303ED8AFE8A0F8B188F40
:1023E0008090880490908904A0908A04B0908B0417
:1023F0004090840450908504609086047090870417
:102400000E9453216B017C01A3019201C501B4011B
:102410000E94D51E9B01AC016D897E898F89988DA4
:102420000E9453219B01AC01C701B6010E94D61E38
:10243000609380047093810480938204909383045A
:1024400080911F03882309F43BC180917C04909103
:102450007D04892B09F45BC080917C0490917D04FC
:10246000019790937D0480937C0480917C049091EB
:102470007D04892B09F0FAC10E94250E0E946F0B82
:1024800080911203813031F466E773E083E594E0D4
:102490000E943B1C80911203823031F46BE773E0A1
:1024A00083E594E00E943B1C6AEA73E083E594E0D4
:1024B0000E943B1C83E594E00E94C40860E08FE02A
:1024C0000E949E1B60E080E10E949E1B60E08DE008
:1024D0000E949E1B80911003882319F08AE80E94B5
:1024E000770B68EC70E080E090E00E94CE1A80915B
:1024F000100381110E94C70980914F0490915004EC
:1025000090938500809384000E941D0EC6C1809127
:102510001203813009F059C06091800470918104E8
:10252000809182049091830420E030E0A9010E9410
:10253000DF2018164CF46091800470918104809122
:102540008204909183040BC0809180049091810457
:10255000A0918204B0918304BC01CD0190582091D8
:1025600090043091910440919204509193040E9400
:10257000DF20181654F560918004709181048091D9
:1025800082049091830420E030E0A9010E94DF20C2
:1025900018164CF48091800490918104A0918204DB
:1025A000B091830409C08091800490918104A0912E
:1025B0008204B0918304B058809390049093910466
:1025C000A0939204B093930448C180911203823087
:1025D00009F04CC1609188047091890480918A044B
:1025E00090918B0420918C0430918D0440918E0445
:1025F00050918F040E94DF2018160CF037C16091B3
:1026000088047091890480918A0490918B042091B0
:1026100013033091140340911503509116030E9447
:10262000D61E60938C0470938D0480938E049093D7
:102630008F0480912A0390912B03209128033091DD
:102640002903821B930B0FEF13E0809FB001819F42
:10265000700D909F700D11247695679580E090E045
:102660000E94082060931B0370931C0380931D033A
:1026700090931E0320912A0330912B03809128030D
:1026800090912903281B390B209FC001219F900D99
:10269000309F900D11249695879525E0289FB001D5
:1026A000299F700D112480E090E00E940820609323
:1026B0001703709318038093190390931A03CDC0E6
:1026C00080911203813009F041C0609180047091C3
:1026D0008104809182049091830420919004309130
:1026E000910440919204509193040E94D51E20E0E1
:1026F00030E0A9010E94DF20181634F460E080E188
:102700000E949E1B61E090C08091800490918104A2
:10271000A0918204B091830420919004309191049F
:102720004091920450919304BC01CD0190580E94B5
:10273000D51E20E030E0A9010E94DF20181634F4F5
:1027400061E080E10E949E1B60E03DC08091120329
:10275000823009F08BC06091880470918904809167
:102760008A0490918B0420918C0430918D044091C7
:102770008E0450918F040E94DF2018160CF076C052
:10278000609188047091890480918A0490918B04EF
:1027900020918C0430918D0440918E0450918F04CF
:1027A0000E94D51E20911703309118034091190300
:1027B00050911A030E94DF2087FD13C061E080E181
:1027C0000E949E1B61E08FE00E949E1B61E08DE0F5
:1027D0000E949E1B80911003882309F445C080E766
:1027E00041C0609188047091890480918A0490911D
:1027F0008B0420918C0430918D0440918E04509173
:102800008F040E94D51E20911B0330911C03409120
:102810001D0350911E030E94DF2087FD12C061E05E
:1028200080E10E949E1B60E08FE00E949E1B61E0A1
:102830008DE00E949E1B809110038823A9F08CE7F5
:1028400011C060E080E10E949E1B61E08FE00E9469
:102850009E1B61E08DE00E949E1B809110038823E7
:1028600019F08AE80E94770B83E003C080917B0413
:10287000815080937B0480917B0481110EC060E0C5
:102880008FE00E949E1B60E080E10E949E1B60E042
:102890008DE00E949E1B0E94C7096C960FB6F894AB
:1028A000DEBF0FBECDBFDF91CF91FF91EF91BF9102
:1028B000AF919F918F917F916F915F914F913F91D8
:1028C0002F911F910F91FF90EF90DF90CF90BF90CD
:1028D000AF909F908F907F906F905F904F903F90C0
:1028E0002F900F900FBE0F901F9018955F926F92D0
:1028F0007F928F929F92AF92BF92CF92DF92EF9290
:10290000FF920F931F93CF93DF9361E088E00E94C3
:10291000651B289862E082E00E94651B61E082E00E
:102920000E949E1B61E08DE00E94651B60E08DE0CF
:102930000E949E1B61E08FE00E94651B60E08FE0BB
:102940000E949E1B61E080E10E94651B60E080E1C7
:102950000E949E1B60E080E00E94651B61E08BE0AE
:102960000E94651B8BE00E94511E68E283E594E0A3
:102970000E940A090E946F0B6091110383E594E0A5
:102980000E94AD0861E070E083E594E00E940008D9
:1029900061E083E594E00E94FA0783E594E00E94F9
:1029A000C40882E00E94D41B90935D0580935C056F
:1029B00080915C0590915D05892B19F481E08093ED
:1029C00048048AE80E94770B64EF71E080E090E0B1
:1029D0000E94CE1A0E94C709EEE4F6E08591949118
:1029E0009093520480935104E6E1F6E0859194912E
:1029F0009093500480934F04EBE3F6E0E491E0936E
:102A00004E04E091FB02F0E0EE0FFF1FEC5FF94F88
:102A10008591949190934D0480934C04E091FA0237
:102A2000F0E0EE0FFF1FE452FA4F859194919093DE
:102A30004B0480934A0480910E0380934904E8ED8F
:102A4000F5E0E491E0931103E1ECF5E085919591D7
:102A5000A591B4918093130390931403A09315034D
:102A6000B09316030E946F0B40E050E060E070E00E
:102A700083E594E00E94F40762EB73E083E594E061
:102A80000E943B1C83E594E00E94C40880E090E033
:102A90000E94C309C82F81E090E00E94C309C53598
:102AA00091F48A3A81F463E080E090E00E94C509E5
:102AB00064E081E090E00E94C50968EC70E080E08D
:102AC00090E00E94CE1A80E090E00E94C309D82FC7
:102AD00081E090E00E94C309C82FD33009F06DC097
:102AE0008CEF8C0F833008F068C082E090E00E9489
:102AF000C3098093FD0283E090E00E94C3098093A4
:102B0000FC0284E090E00E94C3098093FB0285E010
:102B100090E00E94C3098093FA0286E090E00E9450
:102B2000C309809349048BEF8C0F823078F487E0DF
:102B300090E00E94C3098093F902C630E9F488E06E
:102B400090E00E94C3098093F8022CC06091F902C2
:102B500087E090E00E94C50963E080E090E00E9479
:102B6000C50965E081E090E00E94C50968EC70E06D
:102B700080E090E00E94CE1A6091F80288E090E038
:102B80000E94C50963E080E090E00E94C50966E00C
:102B900081E090E00E94C50968EC70E080E090E080
:102BA0000E94CE1A6EEB73E083E594E00E94481C0D
:102BB00083E594E00E94C40858C063EC73E083E5A9
:102BC00094E00E94481C83E594E00E94C40864EFEE
:102BD00071E080E090E00E94CE1A0E946F0B40E00E
:102BE00050E060E070E083E594E00E94F40769E65D
:102BF00073E083E594E00E943B1C83E594E00E942F
:102C0000C4086091FD0282E090E00E94C5096091D5
:102C1000FC0283E090E00E94C5096091FB0284E021
:102C200090E00E94C5096091FA0285E090E00E9460
:102C3000C5096091490486E090E00E94C509609151
:102C4000F90287E090E00E94C5096091F80288E0EF
:102C500090E00E94C50963E080E090E00E94C50911
:102C600066E081E090E00E94C50968EC70E080E0D9
:102C700090E00E94CE1AE091FD02F0E0EE0FFF1FFF
:102C8000E45BF94F859194919093520480935104A1
:102C9000E091FC02F0E0E85CF94FE491E0934E042F
:102CA000E091FB02F0E0EE0FFF1FEC5FF94F859122
:102CB000949190934D0480934C04E091FA02F0E0DB
:102CC000EE0FFF1FE452FA4F8591949190934B04BD
:102CD00080934A04E0914904F0E0E25FFC4F808178
:102CE00080931003E091F902F0E0EB52FA4FE49187
:102CF000E0931103E091F80224E0E29FF001112437
:102D0000EB54FA4F85919591A591B491809313035B
:102D100090931403A0931503B09316030E946F0BB6
:102D200062E083E594E00E94FA076091110383E575
:102D300094E00E94AD0883E594E00E94C408C9E0D5
:102D4000D0E0E0915304F09154040684F785E02D1F
:102D5000E12CF12C0AE210E02EE130E047E050E0F7
:102D600063E270E083E594E0099583E594E00E94D6
:102D7000C40847E050E063E270E083E594E00E941D
:102D8000F4074AE050E0BE0183E594E00E94281D6C
:102D900083E594E00E94C40868EC70E080E090E075
:102DA0000E94CE1A219769F661E083E594E00E94C3
:102DB000FA0783E594E00E94C4080E946F0BCC24BC
:102DC000C394D12C9CE2E92EF12C04E510E02AE515
:102DD00036E040E050E060E070E083E594E00E947F
:102DE000330640E050E060E070E083E594E00E944C
:102DF000F4076AEC73E083E594E00E943B1C6DE20B
:102E000073E083E594E00E943B1C48E250E060E000
:102E100070E083E594E00E94F40763ED73E083E5DE
:102E200094E00E94481C83E594E00E94C4088091CD
:102E300064008E7F8093640080916400846080933E
:102E400064008091640080688093640080916400D5
:102E500082608093640080917A008B7F80937A00F7
:102E600080917A00826080937A0080917A008E7FD0
:102E700080937A0010927C0068EE73E080E090E02E
:102E80000E94CE1A80917A00806480937A008091AB
:102E90007A0086FDFCCF8091780080917900809146
:102EA0007A00806480937A0080917A0086FDFCCF5E
:102EB000809178008091790061E08DE00E949E1BF6
:102EC00061E08FE00E949E1B60E080E10E949E1BFB
:102ED00080911003882319F08AE80E94770B64E63A
:102EE00070E080E090E00E94CE1A60E08FE00E94E7
:102EF0009E1B61E080E10E949E1B8091100388234D
:102F000019F08CE70E94770B64E670E080E090E0B7
:102F10000E94CE1A61E08FE00E949E1B61E080E17A
:102F20000E949E1B80911003882319F080E70E9465
:102F3000770B64E670E080E090E00E94CE1A80910A
:102F4000100381110E94C70960E08FE00E949E1B60
:102F500060E080E10E949E1B60E08DE00E949E1B6D
:102F600064E670E080E090E00E94CE1A82E00E9469
:102F7000D41B90935D0580935C0580915C059091D6
:102F80005D05892B09F0F2C080E090E020912A03D2
:102F900030912B038217930748F4FC01EE0FFF1FBB
:102FA000EC56FB4F118210820196F0CF68EE73E071
:102FB00080E090E00E94CE1ACBE25C2E66246A94F8
:102FC000D3E07D2E1BE2812E912CF894289A86E97D
:102FD00090E00E94F61A289880E090E020912A0361
:102FE00030912B0382179307F8F420917A00206424
:102FF00020937A0020917A0026FDFCCF2091780062
:103000004091790030E0342BFC01EE0FFF1FEC56AD
:10301000FB4F3183208320E030912C03231710F4E1
:103020002F5FFACF0196DACF78940E946F0B80E081
:1030300090E0C2E5D0E020912A0330912B0321508B
:1030400031098217930708F052C06C01AFEFCA1A1A
:10305000DA0AF601EE0FFF1FEC56FB4F408151815B
:1030600020912A0330912B03FC01EE0FFF1FEC5639
:10307000FB4FA080B180E0912A03F0912B03E090F8
:103080005304F0905404549EC001559E900D112499
:10309000B3010E94C8218401061B170B2F5F3F4F0D
:1030A000CE01B9010E94C8219B015A9CC0015B9CC2
:1030B000900D1124B3010E94C8215401A61AB70A29
:1030C000CE01825591093196BF010E94C821D701D6
:1030D0001696ED91FC911797EE24E394F12CA5013F
:1030E00083E594E00995CE5ADF4FC601A4CF83E56E
:1030F00094E00E94C40882E00E94D41B90935D0576
:1031000080935C0580915C0590915D05892B39F079
:103110006AE070E080E090E00E94CE1AECCF61E0BF
:103120008DE00E949E1B64E670E080E090E00E94CB
:10313000CE1A82E00E94D41B90935D0580935C05BB
:1031400080915C0590915D05892B29F46AE070E01F
:1031500080E090E0ECCF64E670E080E090E00E94D8
:10316000CE1A61E08DE00E949E1B2FCF82E00E946C
:10317000D41B90935D0580935C0580915C059091D4
:103180005D05892B99F364E670E080E090E00E9491
:10319000CE1A82E00E94D41B90935D0580935C055B
:1031A00080915C0590915D05892B99F3809148048D
:1031B000882321F0109248040E94840BE091FC02C5
:1031C000F0E0EE0FFF1FE05FF94F8591949190932F
:1031D000500480934F0460914C0470914D0480E042
:1031E00090E00E9408209B01AC0160E070E080E864
:1031F0009FEB0E943E1F0E94AB1F609324037093BD
:103200002503809326039093270360914A047091CD
:103210004B0480E090E00E9408209B01AC0160ED2F
:103220007FE089EC90E40E943E1F20E030E040E81F
:103230005FE30E94D61E9B01AC0160E070E080E875
:103240009FE30E943E1F60932003709321038093AD
:103250002203909323030E946F0B40E050E060E054
:1032600070E083E594E00E94F40769E973E083E588
:1032700094E00E943B1C60915104709152044AE01A
:1032800050E083E594E00E94281D6FED73E083E534
:1032900094E00E943B1C4AE050E060914E0483E5BC
:1032A00094E00E94111D63EE73E083E594E00E94B8
:1032B0003B1C60914C0470914D044AE050E083E562
:1032C00094E00E94281D66EE73E083E594E00E947E
:1032D0003B1C60914A0470914B044AE050E083E546
:1032E00094E00E942E1D6AEE73E083E594E00E9454
:1032F0003B1C80911003882319F062E673E002C042
:1033000065E673E083E594E00E94481C6DEE73E08F
:1033100083E594E00E943B1C4AE050E06091110379
:1033200083E594E00E94111D60EF73E083E594E073
:103330000E943B1C409113035091140360911503AC
:103340007091160322E030E083E594E00E942F1E86
:1033500083E594E00E94C40860ED77E080E090E0AF
:103360000E94CE1A60E08FE00E949E1B60E080E128
:103370000E949E1B60E08DE00E949E1BFE01EE0FEE
:10338000FF1FEC56FB4F118210822196C436D105E7
:10339000A9F7109288041092890410928A0410925E
:1033A0008B0480911203813081F41092800410927A
:1033B000810410928204109283041092900410925F
:1033C000910410929204109293048091120382301F
:1033D00041F410928C0410928D0410928E0410927D
:1033E0008F0410927F0410927E0410927B0488EC6C
:1033F00090E090937D0480937C0481E080931F0390
:103400000E946F0B40E050E060E070E083E594E0E4
:103410000E94F40780911203813031F466E773E073
:1034200083E594E00E943B1C80911203823031F4CA
:103430006BE773E083E594E00E943B1C60E873E077
:1034400083E594E00E943B1C83E594E00E94C4085D
:1034500060E08FE00E949E1B61E080E10E949E1B65
:1034600060E08DE00E949E1BDF91CF911F910F9134
:10347000FF90EF90DF90CF90BF90AF909F908F9094
:103480007F906F905F900C94020E0895EF920F93CF
:103490007AE0E72E09E025E044E063E083E594E08C
:1034A0000E9440080F91EF9008951F920F920FB65F
:1034B0000F9211242F933F938F939F93AF93BF93BA
:1034C00080915F0590916005A0916105B0916205C2
:1034D00030915E0523E0230F2D3720F40196A11DC6
:1034E000B11D05C026E8230F0296A11DB11D209332
:1034F0005E0580935F0590936005A0936105B0938E
:1035000062058091630590916405A0916505B09175
:1035100066050196A11DB11D809363059093640516
:10352000A0936505B0936605BF91AF919F918F9170
:103530003F912F910F900FBE0F901F9018952FB7AE
:10354000F89460915F05709160058091610590919C
:1035500062052FBF08953FB7F8948091630590915D
:103560006405A0916505B091660526B5A89B05C0C8
:103570002F3F19F00196A11DB11D3FBF6627782F7F
:10358000892F9A2F620F711D811D911D42E0660FD8
:10359000771F881F991F4A95D1F70895CF92DF9220
:1035A000EF92FF92CF93DF936B017C010E94AB1AE5
:1035B000EB01C114D104E104F10489F00E94D41E8E
:1035C0000E94AB1A6C1B7D0B683E734090F381E048
:1035D000C81AD108E108F108C851DC4FEACFDF91E1
:1035E000CF91FF90EF90DF90CF90089582309105BA
:1035F00038F0880F991F880F991F05970197F1F7E9
:103600000895789484B5826084BD84B5816084BD5A
:1036100085B5826085BD85B5816085BDEEE6F0E04B
:10362000808181608083E1E8F0E0108280818260A7
:103630008083808181608083E0E8F0E08081816028
:103640008083E1EBF0E0808184608083E0EBF0E058
:10365000808181608083EAE7F0E0808184608083FC
:1036600080818260808380818160808380818068A6
:1036700080831092C1000895833081F028F4813056
:1036800099F08230A1F008958730A9F08830B9F020
:103690008430D1F4809180008F7D03C080918000C0
:1036A0008F7780938000089584B58F7702C084B5AA
:1036B0008F7D84BD08958091B0008F7703C0809185
:1036C000B0008F7D8093B0000895CF93DF9390E09A
:1036D000FC01E258F74F2491FC01EE56F74F84911C
:1036E000882349F190E0880F991FFC01E654F74FB9
:1036F000A591B4918055974FFC01C591D4919FB786
:10370000611108C0F8948C91209582238C93888154
:1037100082230AC0623051F4F8948C91322F309594
:1037200083238C938881822B888304C0F8948C91A6
:10373000822B8C939FBFDF91CF9108950F931F939E
:10374000CF93DF931F92CDB7DEB7282F30E0F9017A
:10375000E659F74F8491F901E258F74F1491F901B6
:10376000EE56F74F04910023C9F0882321F06983B6
:103770000E943C1B6981E02FF0E0EE0FFF1FE05537
:10378000F74FA591B4919FB7F8948C91611103C044
:103790001095812301C0812B8C939FBF0F90DF91E7
:1037A000CF911F910F910895CF93DF93282F30E091
:1037B000F901E659F74F8491F901E258F74FD49196
:1037C000F901EE56F74FC491CC2391F081110E947C
:1037D0003C1BEC2FF0E0EE0FFF1FEA55F74FA591D1
:1037E000B4912C912D2381E090E021F480E002C07F
:1037F00080E090E0DF91CF910895CF92DF92EF9239
:10380000FF920F931F93CF93DF937C016A01EB012B
:1038100000E010E00C151D0571F06991D701ED91E4
:10382000FC910190F081E02DC7010995892B19F0D9
:103830000F5F1F4FEFCFC801DF91CF911F910F9105
:10384000FF90EF90DF90CF9008956115710581F0A2
:10385000DB010D900020E9F7AD0141505109461BF5
:10386000570BDC01ED91FC910280F381E02D09946E
:1038700080E090E008950C94251CDC01ED91FC9112
:103880000190F081E02D099468E374E00C94251C0C
:103890000F931F93CF93DF93EC010E94251C8C01A3
:1038A000CE010E94441C800F911FDF91CF911F9188
:1038B0000F9108958F929F92AF92BF92CF92DF9215
:1038C000EF92FF920F931F93CF93DF93CDB7DEB7A5
:1038D000A1970FB6F894DEBF0FBECDBF7C01C42EFA
:1038E000E52FCB01D22E19A221E02D1510F02AE0F0
:1038F000D22E8E010F5D1F4F8D2C912CA12CB12C3F
:103900006C2D7E2FA50194010E94DC218C2DD29E6E
:1039100080191124015011098A3014F4805D01C00E
:10392000895CF8018083211531054105510521F09D
:10393000C22EE32FCA01E4CFB801C7010E94251CA3
:10394000A1960FB6F894DEBF0FBECDBFDF91CF9129
:103950001F910F91FF90EF90DF90CF90BF90AF90AD
:103960009F908F900895CF92DF92EF92FF920F93E6
:103970001F93CF93DF93EC016A017B012115310581
:1039800079F4E881F9810190F081E02D642FDF91D5
:10399000CF911F910F91FF90EF90DF90CF900994FE
:1039A0002A303105E9F477FF1AC06DE20E943D1C10
:1039B0008C0144275527BA014C195D096E097F090E
:1039C0002AE0CE010E945A1C800F911FDF91CF91F7
:1039D0001F910F91FF90EF90DF90CF9008952AE014
:1039E000B701A601CE01DF91CF911F910F91FF90FA
:1039F000EF90DF90CF900C945A1C2115310541F4C3
:103A0000DC01ED91FC910190F081E02D642F09948F
:103A10000C945A1C9A01462F50E060E070E00C9420
:103A2000FD1C0F931F93CF93DF93EC019A01462F58
:103A300050E060E070E00E94FD1C8C01CE010E940D
:103A4000441C800F911FDF91CF911F910F9108951A
:103A50009A01AB0160E070E00C94FD1C0F931F9382
:103A6000CF93DF93EC019A01AB0160E070E00E941C
:103A7000FD1C8C01CE010E94441C800F911FDF9120
:103A8000CF911F910F9108954F925F926F927F9205
:103A90008F929F92AF92BF92CF92DF92EF92FF925E
:103AA0000F931F93CF93DF93EC016A017B01B22E3A
:103AB0009A01AB01C701B6010E94B621882319F013
:103AC0006BE374E027C026013701E89477F82FEF05
:103AD0003FEF4FE75FE7C301B2010E94B6218111BA
:103AE0000DC02FEF3FEF4FE75FE7C301B2010E9428
:103AF0003A1F18161CF46FE374E00CC02FEF3FEF71
:103B00004FE75FE4C701B6010E94DF201816ACF44E
:103B100063E474E0CE01DF91CF911F910F91FF908C
:103B2000EF90DF90CF90BF90AF909F908F907F905D
:103B30006F905F904F900C94251C2FEF3FEF4FE755
:103B40005FECC701B6010E943A1F87FDE1CF20E07C
:103B500030E0A901C701B6010E943A1F87FF0AC0E1
:103B60006DE2CE010E943D1C8C01F7FAF094F7F84B
:103B7000F09402C000E010E0A12C60E070E080E072
:103B80009FE3AB1441F020E030E040E251E40E94BA
:103B90003E1FA394F6CF9B01AC01C701B6010E9462
:103BA000D61E6B017C010E94DC1F2B013C010E9490
:103BB00008209B01AC01C701B6010E94D51E6B0114
:103BC0007C012AE0B301A201CE010E945A1C080F19
:103BD000191FBB2039F060EB73E0CE010E94251C59
:103BE000080F191F7B2C772041F120E030E040E2E4
:103BF00051E4C701B6010E9453216B017C010E9470
:103C0000D71F4B01AA2497FCA094BA2C2AE030E0DD
:103C1000B501A401CE010E94B31C080F191FC501F4
:103C2000B4010E940A209B01AC01C701B6010E94A9
:103C3000D51E6B017C017A94D6CFC801DF91CF915C
:103C40001F910F91FF90EF90DF90CF90BF90AF90BA
:103C50009F908F907F906F905F904F9008950C94FD
:103C6000441D813039F018F0823051F008951092DF
:103C70006E00089580916F008D7F80936F0008958E
:103C8000809170008D7F8093700081E08093B00000
:103C90008091B100887F84608093B1001092B3005E
:103CA0000895CF93C82F809131038C1307C0E4ECA3
:103CB000F8E084919FEF9093310301C08FEF0E9451
:103CC000311E60E08C2FCF910C949E1B1F920F929F
:103CD0000FB60F9211242F933F934F935F936F93DF
:103CE0007F938F939F93AF93BF93EF93FF938091B5
:103CF0006A0590916B05A0916C05B0916D05892BBB
:103D00008A2B8B2B51F190916705E0916805F0911A
:103D1000690580818927808380916A0590916B0570
:103D2000A0916C05B0916D05181619061A061B06B0
:103D3000C4F480916A0590916B05A0916C05B091D7
:103D40006D050197A109B10980936A0590936B05F0
:103D5000A0936C05B0936D0504C0809131030E945F
:103D6000511EFF91EF91BF91AF919F918F917F91E4
:103D70006F915F914F913F912F910F900FBE0F90D8
:103D80001F9018950E94042208950E94011B0E9412
:103D9000C41E0E947614C0E0D0E00E94451A20970D
:103DA000E1F30E940000F9CF08955058BB27AA27DD
:103DB0000ED0CBC1BCD130F0C1D120F031F49F3F47
:103DC00011F41EF48CC10EF4E095E7FB82C1E92FDB
:103DD000CDD180F3BA17620773078407950718F0EF
:103DE00071F49EF5E5C10EF4E0950B2EBA2FA02DCF
:103DF0000B01B90190010C01CA01A0011124FF2798
:103E0000591B99F0593F50F4503E68F11A16F04092
:103E1000A22F232F342F4427585FF3CF4695379591
:103E20002795A795F0405395C9F77EF41F16BA0B56
:103E3000620B730B840BBAF09150A1F0FF0FBB1F04
:103E4000661F771F881FC2F70EC0BA0F621F731F4D
:103E5000841F48F4879577956795B795F7959E3FAA
:103E600008F0B3CF9395880F08F09927EE0F979538
:103E7000879508950AD108F481E008950CD065C1B2
:103E80005DD140F054D130F021F45F3F19F021C1F1
:103E900051118FC124C16AD198F39923C9F35523D5
:103EA000B1F3951B550BBB27AA276217730784072D
:103EB00038F09F5F5F4F220F331F441FAA1FA9F3E3
:103EC00033D00E2E3AF0E0E830D091505040E695D5
:103ED000001CCAF729D0FE2F27D0660F771F881F36
:103EE000BB1F261737074807AB07B0E809F0BB0B25
:103EF000802DBF01FF2793585F4F2AF09E3F510549
:103F000068F0E7C056C15F3FECF3983EDCF386955E
:103F100077956795B795F7959F5FC9F7880F911DBE
:103F20009695879597F90895E1E0660F771F881FAA
:103F3000BB1F621773078407BA0720F0621B730B5D
:103F4000840BBA0BEE1F88F7E095089519F40EF074
:103F5000C0C02EC1C4C012D1C8F39638C0F707F84C
:103F60000F92E8942BE33AEA48EB5FE7AAD10F926D
:103F70000F920F924DB75EB70F9262D1E2E9F0E077
:103F8000B1D04F915F91EF91FF91E595EE1FFF1F2B
:103F900049F0FE57E0684427EE0F441FFA95E1F719
:103FA0004195550B19D10F9007FE0DC1089504D00E
:103FB0006894B111FEC00895E1D088F09F5790F049
:103FC000B92F9927B751A0F0D1F0660F771F881F3E
:103FD000991F1AF0BA95C9F712C0B13081F0E8D034
:103FE000B1E00895E5C0672F782F8827B85F39F0D2
:103FF000B93FCCF3869577956795B395D9F73EF49D
:1040000090958095709561957F4F8F4F9F4F089544
:10401000E89409C097FB3EF4909580957095619562
:104020007F4F8F4F9F4F9923A9F0F92F96E9BB2718
:104030009395F695879577956795B795F111F8CF94
:10404000FAF4BB0F11F460FF1BC06F5F7F4F8F4FFF
:104050009F4F16C0882311F096E911C0772321F0F5
:104060009EE8872F762F05C0662371F096E8862F8D
:1040700070E060E02AF09A95660F771F881FDAF7E4
:10408000880F9695879597F90895990F0008550F11
:10409000AA0BE0E8FEEF16161706E807F907C0F0CE
:1040A00012161306E407F50798F0621B730B840BD6
:1040B000950B39F40A2661F0232B242B252B21F4B0
:1040C00008950A2609F4A140A6958FEF811D811D50
:1040D000089597F99F6780E870E060E008959FEF8A
:1040E00080EC0895DF93CF931F930F93FF92EF928D
:1040F000DF927B018C01689405C0DA2EEF01DFD0DE
:10410000FE01E894A5912591359145915591AEF325
:10411000EF015DDEFE019701A801DA9479F7DF90E7
:10412000EF90FF900F911F91CF91DF9108950024A0
:104130000A941616170618060906089500240A940C
:1041400012161306140605060895092E0394000C92
:1041500011F4882352F0BB0F40F4BF2B11F460FF21
:1041600004C06F5F7F4F8F4F9F4F089557FD90584A
:10417000440F551F59F05F3F71F04795880F97FB2B
:10418000991F61F09F3F79F08795089512161306E5
:104190001406551FF2CF4695F1DF08C01616170614
:1041A0001806991FF1CF8695710561050894089549
:1041B000E894BB2766277727CB0197F9089565DF39
:1041C00008F48FEF08959B01AC0160E070E080E897
:1041D0009FE354CE7ECFCEC0D1DFE8F39923D9F34D
:1041E000940F511DBBF39150504094F059F0882327
:1041F00032F0660F771F881F91505040C1F79E3FE5
:10420000510544F7880F911D9695879597F9089564
:104210005F3FACF0983E9CF0BB27869577956795FD
:10422000B79508F4B1609395C1F7BB0F58F711F437
:1042300060FFE8CF6F5F7F4F8F4F9F4FE3CFB9CFC6
:10424000FA01DC01AA0FBB1F9B01AC01BF5728F488
:1042500022273327442750781FC0B75188F4AB2F4B
:104260000024469537952795011CA395D2F300208D
:1042700069F0220F331F441FB395DAF30DD095CDAB
:1042800061307105A0E88A07B94630F49B01AC01A2
:104290006627772788279078309621F0208331830E
:1042A0004283538308950BD050CF41DF28F046DF7F
:1042B00018F0952309F00DCF12CF11247ACF56DFD5
:1042C000A0F3959FD1F3950F50E0551F629FF00129
:1042D000729FBB27F00DB11D639FAA27F00DB11D82
:1042E000AA1F649F6627B00DA11D661F829F22270B
:1042F000B00DA11D621F739FB00DA11D621F839F92
:10430000A00D611D221F749F3327A00D611D231F67
:10431000849F600D211D822F762F6A2F11249F57B5
:1043200050408AF0E1F088234AF0EE0FFF1FBB1FD8
:10433000661F771F881F91505040A9F79E3F510577
:1043400070F0C7CE36CF5F3FECF3983EDCF3869536
:1043500077956795B795F795E7959F5FC1F7FE2B22
:10436000880F911D9695879597F908958EDE880B95
:10437000990B08959F3F31F0915020F487957795E0
:104380006795B795880F911D9695879597F908952C
:10439000AA1BBB1B51E107C0AA1FBB1FA617B7076B
:1043A00010F0A61BB70B881F991F5A95A9F7809587
:1043B0009095BC01CD010895A1E21A2EAA1BBB1B4A
:1043C000FD010DC0AA1FBB1FEE1FFF1FA217B307E1
:1043D000E407F50720F0A21BB30BE40BF50B661FF7
:1043E000771F881F991F1A9469F7609570958095BB
:1043F00090959B01AC01BD01CF010895EE0FFF1F09
:104400000590F491E02D099481E090E0F8940C94EB
:104410005422BB274A3031F4992322F4BDE290950F
:1044200081959F4F0C941522BB27FB015527AA2786
:10443000880F991FAA1FA41710F0A41B8395505131
:10444000B9F7A05DAA3308F0A95DA193009779F7A9
:10445000B111B1931192CB010C944422F999FECF82
:1044600092BD81BDF89A992780B50895262FF999B4
:10447000FECF1FBA92BD81BD20BD0FB6F894FA9A47
:10448000F99A0FBE01960895DC01FC01672F719126
:104490007723E1F7329704C07C916D93708362912A
:0C44A000AE17BF07C8F30895F894FFCFD3
:1044AC000000000000000000000000000000000000
:1044BC0000000000000000000000000000000000F0
:1044CC00000000000000C0E0F0F8FCFCFEFFFCE087
:1044DC0000000000000000000000000000000000D0
:1044EC0000000000000000000000000000000000C0
:1044FC0000000000000000000000000000000000B0
:10450C000000000000F8F8F8F8F8F8F8F8F8F8F8F7
:10451C00F8F0F0E0E0C080C0FCFFFFFFFF7F3F7FC2
:10452C00FFFFFFFFFF000000000000000000000084
:10453C00000000000000000000000000000000006F
:10454C00000000000000000000000000000000005F
:10455C00000000000000000000000F1F3F7FFFFF65
:10456C00FFFFFFFFFFFFE7C7C7878F9F9FFFFFFF7F
:10457C00C1C0E0FCFFFFFFFFFFFCFCFCFCFEFEFEED
:10458C00FCFCF8F8F0E0C0C00000000000000000E7
:10459C00000000000000000000000000000000000F
:1045AC0000000000000000000000000000000000FF
:1045BC000080C0E0F1FBFFFFFFFFFF7F1F0F0F87A5
:1045CC00E7FFFFFF1F1F3FF9F8F8F8F8F8F8FDFFB9
:1045DC00FFFFFFFFFFFFFFFF7F3F0F070100000002
:1045EC0000000000000000000000000000000000BF
:1045FC0000000000000000000000000000000000AF
:10460C00000000F0FEFFFFFFFFFFFFFFFFFFFFFEBC
:10461C007E3F3F0F1FFFFFFFFCF0E0F1FFFFFFFFAE
:10462C00FFFCF0010101010101010100000000008B
:10463C00000000000000000000000000000000006E
:10464C00000000000000000000000000000000005E
:10465C000000000000000003030303030303030135
:10466C0001010100000000000000030F1F3F7F7FCD
:10467C00FFFFFFFF7F7F1F03000000000000000012
:10468C00000000000000000000000000000000001E
:10469C000000000000000000030307010301F30306
:1046AC00FD03080415041E0424042D043304010026
:1046BC0001320200007A4400606A4600409C4501C9
:1046CC00DF4F6D3F14AE673F0F00640001332E388F
:1046DC0000FF00000000A007FD1BC21E8E04940505
:1046EC00AB054505C105F605140600000000A00742
:1046FC00FD1B06088E049405AB054505C105F605A2
:10470C0014064F4E004F464600454550524F4D2023
:10471C0057524954450044594E20005354412000EF
:10472C00484541542E2E2E004420005320005A3A66
:10473C000052583A0020443A004C3A00455252205C
:10474C00303100455252203032005A45524F2E2EF5
:10475C002E00454550524F4D2052454144004F2E9E
:10476C004B2E0045525220303000466F787950491C
:10477C0020760028432920466F78794C616200200E
:10478C00523A00493A0020463A00533A00433A0064
:10479C00473A0050554C5345204C454E0050554C13
:1047AC005345204652455100494E544547524154B9
:1047BC004F52204B0046494C544552204B00534F0E
:1047CC00554E4400434F4E545241535400475541AB
:1047DC0052440045584954000D0A006E616E006940
:0847EC006E66006F76660000A6
:00000001FF
